:10000000CEC00000EAC00000E8C00000E6C000006A
:10001000E4C00000E2C00000E0C00000DEC000005C
:10002000DCC00000DAC000000C942E13D6C0000023
:10003000D4C00000D2C00000D0C00000CEC000007C
:10004000CCC00000CAC00000C8C00000C6C000008C
:10005000C4C00000C2C00000C0C00000BEC000009C
:10006000BCC00000BAC00000B8C00000B6C00000AC
:10007000B4C00000B2C00000B0C00000AEC00000BC
:10008000ACC00000AAC00000A8C00000A6C00000CC
:10009000A4C00000A2C0000005010904A101A10242
:1000A000850175089501150026FF008103750195EE
:1000B0001315002501350045010509190129138192
:1000C000027501950D0600FF8103150026FF00054E
:1000D000010901A10075089504350046FF000930AB
:1000E0000931093209358102C005017508952709D2
:1000F0000181027508953009019102750895300952
:1001000001B102C0A1028502750895300901B10252
:10011000C0A10285EE750895300901B102C0A102A7
:1001200085EF750895300901B102C0C009022900A8
:1001300001010080FA090400000203000000092107
:100140001101000122940007050203400001070588
:100150008103400001040309040C035800580058AF
:100160000058000000360359005900590059005941
:1001700000590059005900590059005900590059B7
:1001800000590059005900590059005900590059A7
:10019000005900590059005900590000000011246D
:1001A0001FBECFEFD0E2DEBFCDBF13E0A0E0B1E0D5
:1001B000E8EEFBE200E00BBF02C007900D92A83C06
:1001C000B107D9F714E0A8ECB3E001C01D92A63541
:1001D000B107E1F7F8D00C94F21512CFFB01DC0166
:1001E00004C08D910190801921F441505040C8F70E
:1001F000881B990B0895FB01DC0102C001900D9250
:1002000041505040D8F70895A0E0B0E0EAE0F1E0B6
:100210000C94C5157C01EB018A01690109C0CE016E
:100220002196F6010995F70181937F010150104055
:1002300001151105A1F7CDB7DEB7E8E00C94E11583
:10024000DF92EF92FF920F931F937B018C01FB01D2
:100250000995D82EC8010196F7010995982F8D2D83
:100260001F910F91FF90EF90DF900895A0E0B0E014
:10027000ECE3F1E00C94C515EC017B018A01690106
:1002800009C0CE012196F70161917F01F601099520
:100290000150104001151105A1F7CDB7DEB7E8E018
:1002A0000C94E115DF93CF93CDB7DEB786E090E0F5
:1002B00032D09093BE038093BD0388E090E02BD0B2
:1002C0009093C0038093BF038091BD039091BE03C0
:1002D0002FEF8F3F920731F48BEE93E09093BE03A4
:1002E0008093BD038091BF039091C0032FEF8F3F98
:1002F000920731F482E490E29093C0038093BF03AD
:100300008DE394E020E030E0B90146E050E03AD0DF
:10031000CF91DF910895DF93CF9300D0CDB7DEB7B3
:100320009A83898389819A812DE931E0B90188DF37
:100330000F900F90CF91DF910895DF93CF9300D06E
:10034000CDB7DEB79A838983EFE3F0E08081882F11
:1003500090E0827090700097B9F7E1E4F0E0898155
:100360009A8191838083AFE3B0E0EFE3F0E0808196
:1003700081608C93E0E4F0E080810F900F90CF914A
:10038000DF910895DF93CF9300D000D000D0CDB798
:10039000DEB79A8389837C836B835E834D838981F7
:1003A0009A812B813C814D815E81EDE9F1E0B901BB
:1003B0009F012ADF26960FB6F894DEBF0FBECDBF91
:1003C000CF91DF910895DF93CF93CDB7DEB76E97CE
:1003D0000FB6F894DEBF0FBECDBF64DF12D11E8E04
:1003E0001D8E7BC080E090E0A0E8BFE3898F9A8FEC
:1003F000AB8FBC8F698D7A8D8B8D9C8D20E030E02A
:100400004AE755E40E943015DC01CB018D8B9E8BB1
:10041000AF8BB88F6D897E898F89988D20E030E011
:1004200040E85FE30E94AF1488232CF481E090E061
:100430009C8B8B8B3FC06D897E898F89988D20E046
:100440003FEF4FE757E40E942C1518164CF5698DC5
:100450007A8D8B8D9C8D20E030E040E251E40E944B
:100460003015DC01CB01BC01CD010E94B314DC01CD
:10047000CB019C8B8B8B0FC080E991E09A8B898B91
:1004800089899A890197F1F79A8B898B8B899C8945
:1004900001979C8B8B8B8B899C89009769F714C083
:1004A0006D897E898F89988D0E94B314DC01CB0100
:1004B0009C8B8B8B8B899C89988B8F878F85988958
:1004C0000197F1F7988B8F870E94CC0A0E948314C2
:1004D0008D8D9E8D01969E8F8D8F8D8D9E8D27E0AB
:1004E000803D92070CF47ECF81E0809307011E8E41
:1004F0001D8E7AC080E090E0A0E8BFE38B879C87E8
:10050000AD87BE876B857C858D859E8520E030E03C
:100510004AE755E40E943015DC01CB018F839887B0
:10052000A987BA876F81788589859A8520E030E030
:1005300040E85FE30E94AF1488232CF481E090E050
:100540009E838D833FC06F81788589859A8520E061
:100550003FEF4FE757E40E942C1518164CF56B85BA
:100560007C858D859E8520E030E040E251E40E944C
:100570003015DC01CB01BC01CD010E94B314DC01BC
:10058000CB019E838D830FC080E991E09C838B8398
:100590008B819C810197F1F79C838B838D819E8158
:1005A00001979E838D838D819E81009769F714C08A
:1005B0006F81788589859A850E94B314DC01CB010F
:1005C0009E838D838D819E819A83898389819A817F
:1005D0000197F1F79A838983DFD70E9483148D8D69
:1005E0009E8D01969E8F8D8F8D8D9E8D23E0883EF2
:1005F00092070CF47FCF10920701CED70E9483148C
:10060000FCCFDF93CF930F92CDB7DEB7A4E5B0E078
:10061000E4E5F0E08081877F8C9388E10FB6F89461
:1006200080936000109260000FBE80E8898329816A
:1006300080E090E00FB6F894209361008093610011
:100640000FBE06D00E947B120F90CF91DF910895CC
:10065000DF93CF93CDB7DEB7AAE2B0E0EAE2F0E0F5
:100660008081806F8C93ABE2B0E0EBE2F0E08081C0
:100670008F708C93CF91DF910895DF93CF93CDB797
:10068000DEB780EA06D081E080930001CF91DF9150
:100690000895DF93CF930F92CDB7DEB78983ABE296
:1006A000B0E0EBE2F0E08081982F9F708981892B88
:1006B0008C930F90CF91DF910895DF93CF93CDB7B7
:1006C000DEB780E1E6DFCF91DF910895DF93CF932E
:1006D00000D000D000D0CDB7DEB780E6DADF1C82D4
:1006E00088E090E09E838D8309C08C818F5F8C832E
:1006F0008D819E81880F991F9E838D838D819E8120
:100700008034910590F38C818295807F982F926040
:1007100081E061EC492F0E94B50E982F81E0892776
:10072000882311F080E9B5DF198288E090E09B838F
:100730008A8309C089818F5F89838A819B81880F21
:10074000991F9B838A838A819B818034910590F3D2
:1007500089818295807F982F926082E060EC492F9A
:100760000E94B50E982F81E08927882311F080E937
:1007700090DFA2EEB0E0E2EEF0E0808184608C9346
:1007800026960FB6F894DEBF0FBECDBFCF91DF9196
:100790000895DF93CF93CDB7DEB7C658D0400FB6DC
:1007A000F894DEBF0FBECDBF80914F04282F30E0FC
:1007B00065963FAF2EAF659765968EAD9FAD6597F9
:1007C0008330910509F41FC56596EEADFFAD6597C1
:1007D000E430F10584F465962EAD3FAD6597213088
:1007E000310511F165968EAD9FAD6597823091050B
:1007F00009F46CC592C56596EEADFFAD6597EA301C
:10080000F10509F443C565962EAD3FAD65972B30D4
:10081000310509F41BC565968EAD9FAD659789308E
:10082000910509F47AC479C580914E04813A09F0A2
:1008300074C58091500490915104EEED8D3A9E075D
:10084000C9F5CE0142962DEB33E0B90142E050E00C
:10085000D2DCCE01429602962FEB33E0B90142E0A2
:1008600050E0C9DCCE01429604962DE334E0B90194
:1008700046E050E0C0DCA8EEB0E0E8EEF0E08081B9
:10088000877F8C932091540430915504CE01429679
:10089000B9010E943510E8EEF0E08081898BE8EE26
:1008A000F0E089898B7F8083E8EEF0E089898F779B
:1008B000808333C58091500490915104877F937059
:1008C000F3E0873F9F0709F05AC09E012E5E3F4F1D
:1008D00067963FAF2EAF679785E793E069969FAF26
:1008E0008EAF699790E46A969FAF6A976996EEAD6E
:1008F000FFAD6997008069962EAD3FAD69972F5F78
:100900003F4F69963FAF2EAF69976796EEADFFAD4B
:100910006797008267962EAD3FAD67972F5F3F4F79
:1009200067963FAF2EAF67976A963FAD6A97315093
:100930006A963FAF6A976A968FAD6A978823B1F639
:10094000A8EEB0E0E8EEF0E08081877F8C93209104
:10095000540430915504CE014296B9010E943510DD
:10096000E8EEF0E08081888BE8EEF0E088898B7F0C
:100970008083E8EEF0E088898F778083CEC4809111
:10098000500490915104857F9370E3E0853F9E076A
:1009900009F0AFC0A8EEB0E0E8EEF0E08081877F1C
:1009A0008C938091CA03882309F048C09E012E5E73
:1009B0003F4F6C963FAF2EAF6C9785E393E06E96FA
:1009C0009FAF8EAF6E9790E46F969FAF6F976E96C6
:1009D000EEADFFAD6E9700806E962EAD3FAD6E977B
:1009E0002F5F3F4F6E963FAF2EAF6E976C96EEAD7A
:1009F000FFAD6C9700826C962EAD3FAD6C972F5F6C
:100A00003F4F6C963FAF2EAF6C976F963FAD6F9791
:100A100031506F963FAF6F976F968FAD6F9788236A
:100A2000B1F62091540430915504CE014296B9019B
:100A30000E94351081E08093CA034CC0FE0172967B
:100A4000A196FFAFEEAFA19725EF32E0A3963FAF9F
:100A50002EAFA39730E4A4963FAFA497A396EEAD34
:100A6000FFADA3970080A3962EAD3FADA3972F5F58
:100A70003F4FA3963FAF2EAFA397A196EEADFFAD2C
:100A8000A1970082A1962EAD3FADA1972F5F3F4F5A
:100A9000A1963FAF2EAFA197A4963FADA49731503A
:100AA000A4963FAFA497A4968FADA4978823B1F6E0
:100AB000CE014296029623E434E0B90146E050E0CC
:100AC0009ADB2091540430915504CE014296B9012D
:100AD0000E943510E8EEF0E080818F87E8EEF0E0CC
:100AE0008F858B7F8083E8EEF0E08F858F77808322
:100AF00014C48091500490915104827F9370E3E07C
:100B0000823F9E0709F063C09E012E5E3F4FA6966E
:100B10003FAF2EAFA69785EB92E0A8969FAF8EAF22
:100B2000A89790E4A9969FAFA997A896EEADFFADC0
:100B3000A8970080A8962EAD3FADA8972F5F3F4F96
:100B4000A8963FAF2EAFA897A696EEADFFADA6979D
:100B50000082A6962EAD3FADA6972F5F3F4FA6967B
:100B60003FAF2EAFA697A9963FADA9973150A99652
:100B70003FAFA997A9968FADA9978823B1F6CE016B
:100B8000429604962DE334E0B90146E050E033DBB1
:100B9000A8EEB0E0E8EEF0E08081877F8C932091B2
:100BA000540430915504CE014296B9010E9435108B
:100BB000E8EEF0E080818E87E8EEF0E08E858B7FB6
:100BC0008083E8EEF0E08E858F778083A6C38091E6
:100BD0005004909151048F7E9370E3E08F3E9E0706
:100BE00009F05DC09E012E5E3F4FAB963FAF2EAF2A
:100BF000AB9785E792E0AD969FAF8EAFAD9790E44F
:100C0000AE969FAFAE97AD96EEADFFADAD970080BF
:100C1000AD962EAD3FADAD972F5F3F4FAD963FAF39
:100C20002EAFAD97AB96EEADFFADAB970082AB9616
:100C30002EAD3FADAB972F5F3F4FAB963FAF2EAF83
:100C4000AB97AE963FADAE973150AE963FAFAE97F5
:100C5000AE968FADAE978823B1F680910304898F4D
:100C6000A8EEB0E0E8EEF0E08081877F8C932091E1
:100C7000540430915504CE014296B9010E943510BA
:100C8000E8EEF0E080818D87E8EEF0E08D858B7FE7
:100C90008083E8EEF0E08D858F7780833EC380917E
:100CA0005004909151048E7E9370E3E08E3E9E0737
:100CB00009F05AC09E012E5E3F4FE0963FAF2EAF27
:100CC000E09785E392E0E2969FAF8EAFE29790E4E3
:100CD000E3969FAFE397E296EEADFFADE29700801B
:100CE000E2962EAD3FADE2972F5F3F4FE2963FAFCA
:100CF0002EAFE297E096EEADFFADE0970082E09672
:100D00002EAD3FADE0972F5F3F4FE0963FAF2EAF48
:100D1000E097E3963FADE3973150E3963FAFE3971B
:100D2000E3968FADE3978823B1F6A8EEB0E0E8EE46
:100D3000F0E08081877F8C9320915404309155049A
:100D4000CE014296B9010E943510E8EEF0E08081B4
:100D50008C87E8EEF0E08C858B7F8083E8EEF0E016
:100D60008C858F778083D9C28091500490915104F3
:100D700082709370E3E082309E0709F05AC09E01B2
:100D80002E5E3F4FE5963FAF2EAFE59785EF91E0A2
:100D9000E7969FAF8EAFE79790E4E8969FAFE8970E
:100DA000E796EEADFFADE7970080E7962EAD3FAD3D
:100DB000E7972F5F3F4FE7963FAF2EAFE797E59658
:100DC000EEADFFADE5970082E5962EAD3FADE59720
:100DD0002F5F3F4FE5963FAF2EAFE597E8963FADCB
:100DE000E8973150E8963FAFE897E8968FADE897DF
:100DF0008823B1F6A8EEB0E0E8EEF0E08081877FCE
:100E00008C932091540430915504CE014296B9013F
:100E10000E943510E8EEF0E080818B87E8EEF0E08C
:100E20008B858B7F8083E8EEF0E08B858F778083E6
:100E300074C2809150049091510481709370E3E0EA
:100E400081309E0709F05AC09E012E5E3F4FEA9600
:100E50003FAF2EAFEA9785EB91E0EC969FAF8EAF58
:100E6000EC9790E4ED969FAFED97EC96EEADFFAD6D
:100E7000EC970080EC962EAD3FADEC972F5F3F4F87
:100E8000EC963FAF2EAFEC97EA96EEADFFADEA974A
:100E90000082EA962EAD3FADEA972F5F3F4FEA966C
:100EA0003FAF2EAFEA97ED963FADED973150ED96FF
:100EB0003FAFED97ED968FADED978823B1F6A8EE95
:100EC000B0E0E8EEF0E08081877F8C9320915404BD
:100ED00030915504CE014296B9010E943510E8EEDA
:100EE000F0E080818A87E8EEF0E08A858B7F80835E
:100EF000E8EEF0E08A858F7780830FC280915004FE
:100F00009091510481709270E2E081309E0709F067
:100F10006AC09E012E5E3F4FEF963FAF2EAFEF9718
:100F200085E791E0C158DF4F99838883CF57D04040
:100F300090E4CF57DF4F9883C158D040C158DF4F5E
:100F4000E881F981CF57D0400080C158DF4F288118
:100F50003981CF57D0402F5F3F4FC158DF4F398382
:100F60002883CF57D040EF96EEADFFADEF970082CC
:100F7000EF962EAD3FADEF972F5F3F4FEF963FAF10
:100F80002EAFEF97CF57DF4F3881C158D040315047
:100F9000CF57DF4F3883C158D040CF57DF4F8881BC
:100FA000C158D040882351F6A8EEB0E0E8EEF0E05A
:100FB0008081877F8C932091540430915504CE0119
:100FC0004296B9010E943510E8EEF0E080818987F1
:100FD000E8EEF0E089858B7F8083E8EEF0E089859C
:100FE0008F7780839AC180915004909151048170D1
:100FF0009170E1E081309E0709F071C09E012E5E84
:101000003F4FCE57DF4F39832883C258D04085E306
:1010100091E0CC57DF4F99838883C458D04090E447
:10102000CA57DF4F9883C658D040CC57DF4FE8816E
:10103000F981C458D0400080CC57DF4F28813981D6
:10104000C458D0402F5F3F4FCC57DF4F39832883A0
:10105000C458D040CE57DF4FE881F981C258D04004
:101060000082CE57DF4F28813981C258D0402F5F90
:101070003F4FCE57DF4F39832883C258D040CA57DD
:10108000DF4F3881C658D0403150CA57DF4F3883C0
:10109000C658D040CA57DF4F8881C658D0408823F1
:1010A00021F6A8EEB0E0E8EEF0E08081877F8C9337
:1010B0002091540430915504CE014296B901D5D700
:1010C000E8EEF0E080818887E8EEF0E088858B7FAD
:1010D0008083E8EEF0E088858F7780831EC1A8EEDC
:1010E000B0E0E8EEF0E08081877F8C93CE014296FD
:1010F00080D1CE01429662E370E0B7D7E8EEF0E02F
:1011000080818F83E8EEF0E08F818B7F8083E8EE33
:10111000F0E08F818F77808300C180914E0481320F
:1011200009F0FBC0A8EEB0E0E8EEF0E08081877F38
:101130008C9305C080914D04882309F4EEC0E8EE3D
:10114000F0E08081882F90E084709070009791F398
:101150001E820DC08E81282F30E0E1EFF0E080810B
:10116000F901E350FC4F80838E818F5F8E838E81E7
:10117000282F30E0809154049091550428173907A6
:1011800048F3E8EEF0E080818D83E8EEF0E08D81B9
:101190008B7F8083E8EEF0E08D818F77808340D66F
:1011A0008091500490915104EEED8D3A9E07C1F468
:1011B0008DEF93E026E030E0B90142E050E0B7D097
:1011C0008FEF93E028E030E0B90142E050E0AFD08B
:1011D00081E094E020E030E0B90146E050E0A7D0A3
:1011E0008091500490915104F3E0853F9F0709F0EE
:1011F00094C083E494E02FEF33E0B90146E050E07F
:101200000E94FB008AC080914E04813A09F085C09B
:10121000A8EEB0E0E8EEF0E08081877F8C938091CB
:1012200000018A83E1EFF0E08A818083E8EEF0E05C
:1012300080818C83E8EEF0E08C818E7F8083E8EE05
:10124000F0E08C818F778083EBD567C080914E046E
:10125000813209F062C0A8EEB0E0E8EEF0E08081F3
:10126000877F8C93809150049091510463961FAEB8
:101270006397009721F021E063962FAF6397639601
:101280003FAD639730930001CBD547C080914E04AA
:10129000813209F042C0A8EEB0E0E8EEF0E08081D3
:1012A000877F8C938091500490915104807000242A
:1012B000880F991F001C880F991F001C892F902DE3
:1012C0009093020180930101ABD527C080914E0419
:1012D000813A19F5A8EEB0E0E8EEF0E08081877F72
:1012E0008C93809101019091020196958795969536
:1012F00087958983E1EFF0E089818083E8EEF0E073
:1013000080818B83E8EEF0E08B818E7F8083E8EE36
:10131000F0E08B818F77808383D5CA57DF4F0FB67C
:10132000F894DEBF0FBECDBFCF91DF910895DF935C
:10133000CF9300D000D000D0CDB7DEB79A83898399
:101340007C836B835E834D838B819C8129813A8171
:101350004D815E81E9EBF9E0B9019F010E94360100
:1013600026960FB6F894DEBF0FBECDBFCF91DF91AA
:101370000895DF93CF9300D00F92CDB7DEB79A8355
:1013800089836B83EFE3F0E08081882F90E08270A7
:1013900090700097B9F7EFE3F0E01082E1E4F0E03D
:1013A00089819A8191838083E0E4F0E08B8180835E
:1013B0000FB6F894FA9AF99A0FBE0F900F900F900B
:1013C000CF91DF910895DF93CF93CDB7DEB78091B2
:1013D000C8039091C903009749F08091C803909188
:1013E000C90301979093C9038093C803CF91DF91FC
:1013F0000895DF93CF9300D0CDB7DEB79A8389836A
:1014000089819A8123E031E0B90142E350E00E94F2
:10141000FB000F900F90CF91DF910895DF93CF9352
:101420000F92CDB7DEB789830F90CF91DF910895EA
:10143000DF93CF93CDB7DEB7E9970FB6F894DEBF51
:101440000FBECDBF81E08A83CE010396D2DF8BEC45
:1014500093E09E012D5F3F4FB90142E350E00E94AF
:10146000EE001A82009711F081E08A8380910101D9
:1014700090910201009781F08091C8039091C90377
:10148000009751F480910101909102019093C9035A
:101490008093C80381E08A83E9EEF0E081E08083F5
:1014A000E8EEF0E08081882F90E0807290700097E5
:1014B000B1F18A81882399F18BEC93E09EAB8DABDF
:1014C000FE013396F8AFEFABF2E3F9AFEFA9F8AD59
:1014D00000808FA998AD019698AF8FABEDA9FEA9BA
:1014E00000828DA99EA901969EAB8DAB99AD9150BE
:1014F00099AFE9ADEE2351F7CE01039662E370E0B8
:1015000035D5E8EEF0E080818983E8EEF0E089816E
:101510008E7F8083E8EEF0E089818F778083E99683
:101520000FB6F894DEBF0FBECDBFCF91DF91089507
:10153000DF93CF9300D0CDB7DEB7E9EEF0E082E0E5
:101540008083E8EEF0E08081882F90E084709070D6
:101550000097E9F0E8EEF0E08081882F90E080725B
:101560009070009731F0E1EFF0E080818A838A810A
:1015700055DFE8EEF0E080818983E8EEF0E08981D4
:101580008B7F8083E8EEF0E089818F7780830F90F6
:101590000F90CF91DF910895DF93CF93CDB7DEB752
:1015A00080914D04843011F443DFC2DFCF91DF918D
:1015B0000895DF93CF93CDB7DEB76A970FB6F8944F
:1015C000DEBF0FBECDBF998B888B6A8B5C8B4B8B3C
:1015D0003E8B2D8B88899989892F99278F878889B8
:1015E0008E871D861C861B861A868F85282F30E0E5
:1015F0003A8F298F898D9A8D83309105B1F1298D8C
:101600003A8D243031055CF4898D9A8D81309105B5
:1016100099F0298D3A8D22303105D9F08AC0898D13
:101620009A8D8132910509F46DC0298D3A8D22324F
:10163000310509F473C07DC085EB93E09D878C87ED
:1016400082E190E09B878A87ED89FE8982E0808332
:1016500070C08CE291E09D878C8789E290E09B8747
:101660008A87ED89FE89108264C08E85282F30E03C
:10167000388F2F8B8F89988D81309105E1F02F89DC
:10168000388D2230310549F18F89988D009709F006
:1016900035C085E591E09D878C8785E591E0998748
:1016A0008887E885F98584918F838F81882F90E0E2
:1016B0009B878A8723C089E591E09D878C8789E590
:1016C00091E09E838D83ED81FE8184918C838C815A
:1016D000882F90E09B878A8711C085E691E09D87DF
:1016E0008C8785E691E09B838A83EA81FB818491E4
:1016F00089838981882F90E09B878A87ED89FE897D
:10170000108217C08EE391E09D878C8789E090E07E
:101710009B878A87ED89FE8910820BC088E990E05B
:101720009D878C8784E990E09B878A87ED89FE8975
:101730001082EB89FC898C859D85918380838A85C5
:101740009B856A960FB6F894DEBF0FBECDBFCF91D2
:10175000DF910895DF93CF93CDB7DEB727970FB60C
:10176000F894DEBF0FBECDBF1D828EE494E09C8353
:101770008B8319820EC0E1EFF0E08081EB81FC8168
:1017800080838B819C8101969C838B8389818F5F71
:1017900089838981883078F380914E048A8380918F
:1017A0004F04282F30E03F832E838E819F81853028
:1017B0009105C1F12E813F81263031057CF48E8167
:1017C0009F818130910521F12E813F8123303105A8
:1017D000F9F08E819F81009789F042C02E813F8170
:1017E0002830310581F18E819F818930910591F1F9
:1017F0002E813F8126303105E1F032C08A81803868
:1018000019F08A81823861F5BED181E08D8328C0CC
:101810008A81882319F08A81823011F521D281E0F2
:101820008D831EC08A818823D9F441D081E08D83C5
:1018300017C08A81803819F08A81813889F442D1B1
:1018400081E08D830DC08A81803851F48BD081E096
:101850008D8306C08A81882319F459D081E08D8355
:101860008D8191E08927882311F00E94C903E8EE59
:10187000F0E08081882F90E088709070009771F080
:10188000ABEEB0E0EBEEF0E0808180628C93A8EEEE
:10189000B0E0E8EEF0E08081877F8C9327960FB66A
:1018A000F894DEBF0FBECDBFCF91DF910895DF93D7
:1018B000CF930F92CDB7DEB7809150049091510431
:1018C0008F778983A8EEB0E0E8EEF0E08081877F33
:1018D0008C93A6D204C080914D048823A1F0E8EE39
:1018E000F0E08081882F90E081709070009799F3EC
:1018F0008981882319F083E080934D04E3EEF0E0C2
:101900008981806880830F90CF91DF910895DF9364
:10191000CF930F92CDB7DEB78091500490915104D0
:101920008230E0F4A8EEB0E0E8EEF0E08081877F5E
:101930008C93809150049091510480934B0470D209
:1019400080914B04882319F084E0898302C083E0EE
:101950008983898180934D040E9466030F90CF9103
:10196000DF910895DF93CF9300D0CDB7DEB7A8EE17
:10197000B0E0E8EEF0E08081877F8C9380914B04AB
:101980008983E1EFF0E089818083E8EEF0E08081F7
:101990008A83E8EEF0E08A818E7F8083E8EEF0E0D3
:1019A0008A818F7780833CD20F900F90CF91DF9107
:1019B0000895DF93CF9300D0CDB7DEB789838981B7
:1019C0008F70805D898389818A3328F08981982F7F
:1019D000995F9A8302C089818A838A810F900F90D0
:1019E000CF91DF9108950F931F93DF93CF93CDB7DE
:1019F000DEB7E1970FB6F894DEBF0FBECDBF83E030
:101A000089878AE288878EE08F831E8233C08F8128
:101A1000882F90E09C838B8381E2EB81FC81809313
:101A2000570084918A838A818D838E81882F90E0EC
:101A300081709070882339F08D8182958F708D83AD
:101A40008F818F5F8F838E81082F10E08D81B1DFB2
:101A5000482F50E0C80101969C01220F331FCE0190
:101A60000196820F931FFC013796518340838E812C
:101A70008F5F8E838E81843150F2A8EEB0E0E8EE65
:101A8000F0E08081877F8C93CE0108966AE270E057
:101A9000ECD2E8EEF0E080818983E8EEF0E0898125
:101AA0008B7F8083E8EEF0E089818F778083E196F9
:101AB0000FB6F894DEBF0FBECDBFCF91DF911F915F
:101AC0000F910895DF93CF9300D000D000D0CDB711
:101AD000DEB7809150049091510423E08C3D920731
:101AE00011F481DF47C0409150045091510480911E
:101AF000520490915304682F9E012C5F3F4FFE01CA
:101B00003696CA01A9019F0154DD9B838A838A818D
:101B10009B81009779F1A8EEB0E0E8EEF0E08081DB
:101B2000877F8C938E81882339F48C819D812A81D3
:101B30003B81B90159D310C08E81813039F48C8139
:101B40009D812A813B81B90115D406C08C819D817C
:101B50002A813B81B90189D2E8EEF0E08081898356
:101B6000E8EEF0E089818B7F8083E8EEF0E0898108
:101B70008F77808326960FB6F894DEBF0FBECDBF59
:101B8000CF91DF910895DF93CF9300D000D000D0A4
:101B9000CDB7DEB71C8280914E04282F30E03E8303
:101BA0002D838D819E818038910531F02D813E817C
:101BB0002238310581F04BC080914904882319F007
:101BC0008C8181608C8380914A048823D1F08C8140
:101BD00082608C8316C0E9EEF0E08091520490910F
:101BE00053048083EBEEF0E08081882F90E08072D8
:101BF00090701C82009711F081E08C83E9EEF0E098
:101C00001082A8EEB0E0E8EEF0E08081877F8C9350
:101C10008C81882F90E09A838983E1EFF0E08981BD
:101C20008083E1EFF0E089819A81892F9927808371
:101C3000E8EEF0E080818B83E8EEF0E08B818E7F30
:101C40008083E8EEF0E08B818F778083E9D0269661
:101C50000FB6F894DEBF0FBECDBFCF91DF910895D0
:101C6000DF93CF9300D000D0CDB7DEB780914E0484
:101C7000882F90E09C012F7130703C832B838B81E7
:101C80009C81009731F02B813C812230310599F005
:101C900065C08091500490915104813009F05EC07C
:101CA00080914F041A82833011F431E03A838A81A3
:101CB00080934A0448C08091500490915104882335
:101CC00009F041C080915204909153048770898338
:101CD0008981882309F442C0E9EEF0E0898180839C
:101CE000EBEEF0E08081882F90E081709070882387
:101CF00051F180914F04833041F4ABEEB0E0EBEE54
:101D0000F0E0808180628C931EC0ABEEB0E0EBEE21
:101D1000F0E0808180618C93EAEEF0E08981282FE9
:101D200030E081E090E002C0880F991F2A95E2F729
:101D30008083EAEEF0E01082ABEEB0E0EBEEF0E094
:101D4000808188608C93E9EEF0E01082A8EEB0E02C
:101D5000E8EEF0E08081877F8C9362D00F900F9047
:101D60000F900F90CF91DF910895DF93CF9300D024
:101D700000D0CDB7DEB789836A834B83E9EEF0E00C
:101D800089818083ABEEB0E0EBEEF0E08081816092
:101D90008C93EDEEF0E01082ECEEF0E08A8180832F
:101DA000EDEEF0E08B818083EEEEF0E080811C822E
:101DB000882314F481E08C838C810F900F900F9016
:101DC0000F90CF91DF910895DF93CF930F92CDB70E
:101DD000DEB7E4EFF0E0108219821BC0E9EEF0E01C
:101DE00089818083E0EFF0E01082E8EEF0E010827D
:101DF000ADEEB0E0EDEEF0E080818D7F8C93ABEE48
:101E0000B0E0EBEEF0E080818E7F8C9389818F5F74
:101E100089838981873010F30F90CF91DF910895E6
:101E2000DF93CF9300D0CDB7DEB780914E048823E7
:101E30000CF504C080914D04882399F1E8EEF0E0A0
:101E40008081882F90E084709070009799F3E8EE7D
:101E5000F0E080818A83E8EEF0E08A818B7F8083E6
:101E6000E8EEF0E08A818F7780831BC080914D047B
:101E70008823B9F0E8EEF0E08081882F90E081704F
:101E80009070009799F3E8EEF0E080818983E8EEA6
:101E9000F0E089818E7F8083E8EEF0E089818F77A2
:101EA00080830F900F90CF91DF910895DF93CF93B0
:101EB00000D00F92CDB7DEB784E68983ECEEF0E078
:101EC0008081882F90E081709070882359F0E8EE2F
:101ED000F0E08081882F90E081709070882369F015
:101EE0001B823DC0E8EEF0E08081882F90E0847096
:101EF0009070009711F01B8232C080914D048823AE
:101F000019F482E08B832BC0EBEEF0E08081882F08
:101F100090E080729070009719F081E08B831FC071
:101F2000E1EEF0E08081882F90E08470907000975F
:101F300029F2A1EEB0E0E1EEF0E080818B7F8C939E
:101F40001A828981882311F481E08A8389818150F2
:101F500089838A81882309F4B1CF83E08B838B81C5
:101F60000F900F900F90CF91DF910895DF93CF9353
:101F7000CDB7DEB72A970FB6F894DEBF0FBECDBF40
:101F80009F838E83798768878E819F819D838C83D1
:101F90008DDF8B838B818823A1F18B818A8736C06B
:101FA000E8EEF0E08081882F90E0807290700097DA
:101FB000B1F4E8EEF0E080818A83E8EEF0E08A8117
:101FC0008E7F8083E8EEF0E08A818F7780836EDFFA
:101FD0008B838B818823A9F08B818A8717C0EC8142
:101FE000FD8120818C819D8101969D838C83298335
:101FF000E1EFF0E089818083888599850197998751
:10200000888788859985009759F61A868A852A9641
:102010000FB6F894DEBF0FBECDBFCF91DF9108950C
:10202000DF93CF9300D0CDB7DEB79A838983EFE3F8
:10203000F0E08081882F90E0827090700097B9F76F
:10204000E1E4F0E089819A8191838083AFE3B0E09D
:10205000EFE3F0E0808181608C93E0E4F0E0808148
:102060000F900F90CF91DF910895DF93CF93CDB76D
:10207000DEB72D970FB6F894DEBF0FBECDBF9A879F
:1020800089877C876B8789859A8598878F831E824D
:1020900020915404309155048B859C85281739076D
:1020A00038F480915404909155049C878B8777C0B5
:1020B0008B859C85009709F072C0E8EEF0E0808186
:1020C0008D83E8EEF0E08D818E7F8083E8EEF0E096
:1020D0008D818F77808363C0E8EEF0E08081882F68
:1020E00090E088709070009719F081E08D8772C041
:1020F000E8EEF0E08081882F90E084709070009787
:1021000009F05EC080914D04882319F482E08D8728
:1021100061C0E8EEF0E08081882F90E081709070DF
:102120008823E9F1E2EFF0E0808191819C838B8349
:1021300017C0EF81F88520818F8198850196988757
:102140008F832983E1EFF0E0898180838B859C85F3
:1021500001979C878B878B819C8101969C838B83C5
:102160008B859C85009729F08B819C81803491051B
:1021700000F31E828B819C818034910511F481E0F3
:102180008E83E8EEF0E080818A83E8EEF0E08A81D9
:102190008E7F8083E8EEF0E08A818F7780838B8565
:1021A0009C85009709F098CF8E81882309F094CF01
:1021B00007C080914D04882319F482E08D870AC0FE
:1021C000E8EEF0E08081882F90E0847090700097B6
:1021D00081F31D868D852D960FB6F894DEBF0FBE58
:1021E000CDBFCF91DF910895DF93CF93CDB7DEB709
:1021F00060970FB6F894DEBF0FBECDBF9D878C876A
:102200007F876E878C859D859B878A87198620911D
:102210005404309155048E859F852817390738F46A
:1022200080915404909155049F878E877EC08E853F
:102230009F85009709F079C0E8EEF0E080818887FB
:10224000E8EEF0E088858E7F8083E8EEF0E0888518
:102250008F7780836AC0E8EEF0E08081882F90E07D
:1022600088709070009719F081E0888B79C0E8EE53
:10227000F0E08081882F90E084709070009709F0E2
:1022800065C080914D04882319F482E0888B68C072
:10229000E8EEF0E08081882F90E0817090708823D4
:1022A00009F443C0E2EFF0E0808191819F838E8347
:1022B0001DC08A859B859D838C838A859B8501961D
:1022C0009B878A87EC81FD8184918B838B818983B5
:1022D000E1EFF0E0898180838E859F8501979F875C
:1022E0008E878E819F8101969F838E838E859F85A9
:1022F000009729F08E819F8180349105D0F2198654
:102300008E819F818034910511F481E08987E8EE08
:10231000F0E080818A83E8EEF0E08A818E7F80831E
:10232000E8EEF0E08A818F7780838E859F85009725
:1023300009F091CF8985882309F08DCF07C080915E
:102340004D04882319F482E0888B0AC0E8EEF0E09F
:102350008081882F90E084709070009781F3188AB4
:10236000888960960FB6F894DEBF0FBECDBFCF91BF
:10237000DF910895DF93CF93CDB7DEB72D970FB6DA
:10238000F894DEBF0FBECDBF9A8789877C876B87A5
:1023900089859A8598878F831E8220915404309175
:1023A00055048B859C852817390738F4809154048F
:1023B000909155049C878B8779C08B859C8500976D
:1023C00009F074C0E8EEF0E080818D83E8EEF0E083
:1023D0008D818E7F8083E8EEF0E08D818F77808322
:1023E00065C0E8EEF0E08081882F90E08870907002
:1023F000009719F081E08D8774C0E8EEF0E08081ED
:10240000882F90E084709070009709F060C08091F0
:102410004D04882319F482E08D8763C0E8EEF0E074
:102420008081882F90E081709070882309F43EC0ED
:10243000E2EFF0E0808191819C838B8318C02F8133
:1024400038858F819885019698878F83C901E8DD4B
:102450008983E1EFF0E0898180838B859C850197FA
:102460009C878B878B819C8101969C838B838B853A
:102470009C85009729F08B819C8180349105F8F22E
:102480001E828B819C818034910511F481E08E83C2
:10249000E8EEF0E080818A83E8EEF0E08A818E7FCA
:1024A0008083E8EEF0E08A818F7780838B859C853E
:1024B000009709F096CF8E81882309F092CF07C04C
:1024C00080914D04882319F482E08D870AC0E8EEDC
:1024D000F0E08081882F90E084709070009781F305
:1024E0001D868D852D960FB6F894DEBF0FBECDBF2D
:1024F000CF91DF910895DF93CF93CDB7DEB7A7EDEE
:10250000B0E0E7EDF0E0808180688C930ED0A8ED1C
:10251000B0E0E8EDF0E0808180618C9381E0809311
:102520004C047894CF91DF910895DF93CF930F926D
:10253000CDB7DEB775D085D010924D0410924B0404
:1025400010924A0410924904E9E4F0E084E18083A7
:10255000A9E4B0E0E9E4F0E0808182608C93E9E4F2
:10256000F0E08081882F90E0817090700097B9F33F
:10257000E8EDF0E080818983E8EDF0E089818F77F4
:102580008083E8EDF0E0898180688083A7EDB0E08A
:10259000E7EDF0E0808181608C93A8EDB0E0E8ED9C
:1025A000F0E080818F7D8C93A0EEB0E0E0EEF0E073
:1025B00080818B7F8C93A0EEB0E0E0EEF0E0808134
:1025C0008E7F8C93A1EEB0E0E1EEF0E080818E7F13
:1025D0008C93A2EEB0E0E2EEF0E0808181608C931B
:1025E000A1EEB0E0E1EEF0E08081877F8C93A2EE77
:1025F000B0E0E2EEF0E0808188608C93A8EDB0E07E
:10260000E8EDF0E0808181608C930F90CF91DF91B5
:102610000895DF93CF93CDB7DEB7CF91DF910895C3
:10262000DF93CF93CDB7DEB7A8EDB0E0E8EDF0E0F3
:1026300080818C7F8C93E2EEF0E01082CF91DF916D
:102640000895DF93CF93CDB7DEB7EAEDF0E01082C7
:10265000E1EEF0E01082CF91DF9108951F920F928A
:102660000FB60F9200905B000F9211242F933F93AF
:102670004F935F936F937F938F939F93AF93BF938A
:10268000EF93FF93DF93CF9300D000D0CDB7DEB7A9
:10269000EAEDF0E08081882F90E0817090708823CF
:1026A00019F1E8EDF0E08081882F90E08170907062
:1026B0008823D1F0AAEDB0E0EAEDF0E080818E7FD2
:1026C0008C93E9EDF0E08081882F90E0817090702C
:1026D000882331F081E080934D040E943D0304C0C3
:1026E00010924D040E945D03E1EEF0E08081882F9E
:1026F00090E081709070882361F1E2EEF0E08081DB
:10270000882F90E081709070882319F1A1EEB0E0DD
:10271000E1EEF0E080818E7F8C93A2EEB0E0E2EEFD
:10272000F0E080818E7F8C93A2EEB0E0E2EEF0E0EC
:10273000808180618C93A8EDB0E0E8EDF0E08081CD
:1027400080628C93E9E4F0E0108285E080934D0490
:1027500060DFE1EEF0E08081882F90E08071907082
:10276000009709F447C0E2EEF0E08081882F90E006
:1027700080719070009709F43DC0E9E4F0E084E1D5
:102780008083A9E4B0E0E9E4F0E0808182608C938A
:10279000E9E4F0E08081882F90E0817090700097EC
:1027A000B9F3A8EDB0E0E8EDF0E080818F7D8C9387
:1027B000A1EEB0E0E1EEF0E080818F7E8C93A2EE9E
:1027C000B0E0E2EEF0E080818F7E8C93A2EEB0E08C
:1027D000E2EEF0E0808181608C9380914B0488234D
:1027E00019F084E08C8302C083E08C838C81809319
:1027F0004D040FDFE1EEF0E08081882F90E08870DB
:102800009070009709F44AC0E2EEF0E08081882FD2
:1028100090E088709070009709F440C0A1EEB0E09D
:10282000E1EEF0E08081877F8C9382E080934D041D
:1028300010924B04A1EEB0E0E1EEF0E080818E7FDB
:102840008C93A2EEB0E0E2EEF0E080818E7F8C937C
:10285000A2EEB0E0E2EEF0E0808180618C93B4DA29
:10286000198288E090E09B838A8309C089818F5F09
:1028700089838A819B81880F991F9B838A838A81A0
:102880009B818034910590F389818295807F982F78
:10289000926080E060E0492F68DABBDEE1EEF0E0B4
:1028A0008081882F90E084709070009791F0E2EE24
:1028B000F0E08081882F90E084709070009749F05C
:1028C000A1EEB0E0E1EEF0E080818B7F8C930E947E
:1028D000E3090F900F900F900F90CF91DF91FF9130
:1028E000EF91BF91AF919F918F917F916F915F9188
:1028F0004F913F912F910F9000925B000F900FBE70
:102900000F901F901895DF93CF93CDB7DEB703D00C
:10291000CF91DF910895DF93CF930F92CDB7DEB7BC
:1029200080914D048823B9F0E9EEF0E08081877052
:102930008983E9EEF0E01082E8EEF0E08081882FF4
:1029400090E088709070009711F00E94AA0BE9EE59
:10295000F0E0898180830F90CF91DF9108952FD08F
:1029600008F481E0089557D088F09F5790F0B92F70
:102970009927B751A0F0D1F0660F771F881F991FD4
:102980001AF0BA95C9F712C0B13081F05ED0B1E04B
:1029900008955BC0672F782F8827B85F39F0B93F5B
:1029A000CCF3869577956795B395D9F73EF49095D6
:1029B0008095709561957F4F8F4F9F4F0895990F28
:1029C0000008550FAA0BE0E8FEEF16161706E807F9
:1029D000F907C0F012161306E407F50798F0621B1A
:1029E000730B840B950B39F40A2661F0232B242BEF
:1029F000252B21F408950A2609F4A140A6958FEF0E
:102A0000811D811D089557FD9058440F551F59F0A1
:102A10005F3F71F04795880F97FB991F61F09F3FCB
:102A200079F087950895121613061406551FF2CFF4
:102A30004695F1DF08C0161617061806991FF1CF44
:102A400086957105610508940895E894BB2766276B
:102A50007727CB0197F90895B2DF08F48FEF089537
:102A60000BD078C069D028F06ED018F0952309F00B
:102A70005AC05FC01124EACFC6DFA0F3959FD1F3FF
:102A8000950F50E0551F629FF001729FBB27F00D1C
:102A9000B11D639FAA27F00DB11DAA1F649F662771
:102AA000B00DA11D661F829F2227B00DA11D621FC0
:102AB000739FB00DA11D621F839FA00D611D221F7A
:102AC000749F3327A00D611D231F849F600D211D5E
:102AD000822F762F6A2F11249F5750408AF0E1F001
:102AE00088234AF0EE0FFF1FBB1F661F771F881F4A
:102AF00091505040A9F79E3F510570F014C0A6CFE9
:102B00005F3FECF3983EDCF3869577956795B79534
:102B1000F795E7959F5FC1F7FE2B880F911D96955E
:102B2000879597F9089597F99F6780E870E060E0CE
:102B300008959FEF80EC089500240A941616170656
:102B400018060906089500240A941216130614069E
:102B500005060895092E0394000C11F4882352F001
:102B6000BB0F40F4BF2B11F460FF04C06F5F7F4FB9
:102B70008F4F9F4F08952F923F924F925F926F9287
:102B80007F928F929F92AF92BF92CF92DF92EF92FD
:102B9000FF920F931F93CF93DF93CDB7DEB7CA1B7E
:102BA000DB0B0FB6F894DEBF0FBECDBF09942A88A9
:102BB000398848885F846E847D848C849B84AA8451
:102BC000B984C884DF80EE80FD800C811B81AA81DE
:102BD000B981CE0FD11D0FB6F894DEBF0FBECDBFA9
:082BE000ED010895F894FFCF08
:102BE80001F4010100000000007A80827D000000ED
:102BF80000000000000000000000000000000000CD
:102C080002EE100000000002FF770180021F02029E
:102C1800019C00050000000000000080808080000A
:102C2800000000000000000000000000000000009C
:102C3800000003EE1000000000025477018001FF3D
:102C480001FF01FF01FF000000000000000000007C
:102C58000000000000000000000000000000001E4E
:102C6800FF27103232FF27103232FF27103232FF8F
:102C780027103232000000000000000000000000B1
:102C8800000000000000000000000000000000003C
:102C9800000000000000010300040C0102181818CD
:102CA80018090A10111213000000000400020202A1
:102CB80002000000040404040000010600000000F3
:102CC80000000000000000000000000000000000FC
:102CD80000000000000002010004000000000000E5
:102CE80000000000000000000000000000000000DC
:102CF80000000000000000000000000000000000CC
:102D0800000000000000FFFFFFFFFFFFFFFFFFFFC5
:102D1800FFFFFFFFFF00EE020004EE1000000000BE
:102D280002030801D20000020202000300000200B0
:102D38000002620102015E00320000000000000093
:102D4800000000000000000000000000000000007B
:102D5800000000000000EF0300040301B0000000C1
:102D68000000000000000205019202020191020524
:102D7800019102040076000000000000000000003D
:102D88000000000000030000000000000000000038
:102D98000000000000F2FFFF00000000000000003B
:102DA800035081D8018A0000016419010064000100
:102DB800900019FE00000000000000000000000064
:102DC80000000000000300000000000000000000F8
:102DD80000000000000100000000000000231E00A9
:102DE800035081D8018A00000164190100640001C0
:102DF800900019FE00000000000000000000000024
:102E080000000000000300000000000000000000B7
:102E180000000000000100AAAAAAAAAAAA231E006C
:102E2800035081D8018A000001641901006400017F
:102E3800900019FE000000000000000000000000E3
:102E48000000000000030000000000000000000077
:102E5800000000000001000803D201EEFF1002008C
:102E6800035081D8018A000001641901006400013F
:102E7800900019FE000000000000000000000000A3
:102E88000000000000030000000000000000000037
:102E980000000000001201000200000040000000D5
:082EA80000000101020001001D
:00000001FF
